:020000040800F2
:10500000401C0020D55000089D90000877860008BD
:105010000000000000000000000000000000000090
:10502000000000000000000000000000A5A0000833
:1050300000000000000000006D9B0008E1A10008D6
:10504000E7500008E7500008E7500008E750000864
:10505000E7500008255C0008E7500008E75000080A
:1050600000000000E7500008315B0008E75000082E
:10507000E7500008AD8B000800000000E750000872
:1050800000000000E75000080000000000000000E1
:10509000E750000800000000E7500008E750000853
:1050A000E7500008E7500008E750000879AC000816
:1050B000E7500008E7500008000000000000000072
:1050C0000348854600F07EFC0048004779BD000893
:1050D000401C00200448804704480047FEE7FEE7E4
:1050E000FEE7FEE7FEE7FEE7A1A20008C1500008C8
:1050F00030B50B46014600202022012409E00D4670
:10510000D5409D4205D31D469540491B25469540F7
:1051100040191546521E002DF1DC30BD70B500243B
:105120002546002801DA01244042002901DA012540
:105130004942FFF7DDFFAC4200D04042002C00D0D6
:10514000494270BDF0B51FB40646002082B0054646
:105150004024019100901BE0019922460F46304601
:1051600000F06CFB049A059B801A994110D31046FD
:105170001946224600F052FB361A8F41019722460B
:1051800001200021009F00F049FB38184D4100909C
:105190002046641E0028DFDC019B00982946324629
:1051A00007B0F0BD03460B439B0703D009E008C9D5
:1051B000121F08C0042AFAD203E00B780370401CC7
:1051C000491C521EF9D27047D2B201E00270401C55
:1051D000491EFBD270470022F6E710B513460A4677
:1051E00004461946FFF7F0FF204610BD30B50446CF
:1051F0000020034600E05B1C934203D2E05CCD5CE0
:10520000401BF8D030BDF8B502464A40D40F4200EA
:105210004B0052085B089A4202D2024608461146E9
:105220004A0023D0C30D4A00DDB2120EAD1A202D64
:1052300035DA49020126490AF6058A19002C00D000
:10524000524220214F1B1146B9402A411018C20D6D
:105250009A4221D0002C17D0012D08DCDA05801AE3
:10526000D20F8019D207DBB200F014FBF8BDDA05CB
:10527000801A012340001B06C01880185A4280186B
:10528000CA0F1043490007E04908C2071143DA0575
:10529000801A80194008801800F0F4FAF8BD610007
:1052A0000122511A001BF7E70122D2075140AAE759
:1052B0000122D2075040A6E770B502464A40D50FFA
:1052C00040004A00ED0740085208002814D0002A88
:1052D00012D0C40DD30D41020120C0055202490A6B
:1052E000520AE41A091812187D34914201D3641C41
:1052F00000E04900002C01DA002070BD002391423B
:1053000001D3891A0343400849000028F7D1002936
:105310000AD0914202D10121C90705E0914201D290
:10532000012101E00121C943E005C018401900F046
:10533000A9FA70BDF0B507460846584087B0C00FBF
:10534000049048000E46590040084908BC1A88419C
:1053500005D2384631461E4617460B4602465800CF
:10536000400810434CD0300D039040055900400DCB
:10537000490D0590401A0290402872DA1803012165
:10538000000B09050843019004980092002805D0FD
:1053900001995242002088410092019002984021D8
:1053A0000A1A0199009800F039FA05460C466B4636
:1053B00007CB00F054FAC0197141039A0E0D002377
:1053C000D71756401A467A40164344D0049A002A0A
:1053D0002DD0029A012A039A15DC1205C01A9141B8
:1053E00001263605001C7141D20F059ED20700939D
:1053F000019202962A46234600F092FA07B0F0BDC9
:1054000038463146FAE71605224A0F46B218C01A46
:10541000B74101210905001C4F4100187F41114689
:1054200018187941E20F10436D19644113E0E20747
:105430006D0815436408C2071443039A0126120538
:10544000C01A91413605001C7141CE074008304317
:105450004908C01851412A46234600F054FACDE7C6
:10546000FFE7049801224000C117121A00238B4164
:1054700004983146C417381AA141EEE730B401242C
:10548000E407634030BC55E730B40124E4076140D1
:1054900030BC4FE70000E0FFF0B51FB488B00B99B7
:1054A0000998002448400999C00F4900490809910A
:1054B000C0070B990090490049080B910999089879
:1054C000A64608431CD00B990A98084318D009989F
:1054D00001244000420D4800410D099824050003B5
:1054E000000B204309900B980003000B20430B9006
:1054F00050181C494018002201901446104605E03F
:10550000002001460DB0F0BD032801DA034600E09B
:1055100003239C46C11A0AAE0AE05F0008ADED5BAA
:105520004F00F75B7D430027AA187C41491C5B1E96
:105530006145F2DD410004AB5A522104120C0A43CA
:10554000240C401C0828DFDB01980290009970466B
:1055500001910090059B049A0799069800F0E0F9E4
:10556000D0E700000DFCFFFFF0B50C465C4085B0B5
:10557000E40FE40703944C000026640859009446A5
:10558000490802460296224321D062460A431ED0B1
:105590006200570D4A000E032303550D01240246F5
:1055A0002C492405781B1B0B360B4018234326433C
:1055B000614600901C46501AB44103D30098401C29
:1055C000009002E0921800985B41002803DA002066
:1055D000014605B0F0BD00200121090507468646B9
:1055E00011E064461D46141BB54106D36546521BA7
:1055F000B341744607430C43A646CD07400849080B
:10560000284392185B4105460D43EAD110461843E2
:1056100013D06046194650407140084306D060469A
:10562000101AB34106D20122002306E00022012312
:10563000DB0702E00122D2435310009874460105B3
:10564000381C6141029C039D0019694100F05BF91F
:10565000BFE70000FD030000C217C10F504010B5A6
:105660004018CA079623002100F014F910BD10B5A8
:1056700000229623114600F00DF910BD0EB5C21799
:10568000C10F5040CA0740180021054B02930192F8
:1056900000910A460B4600F043F903B000BD00003C
:1056A000330400000EB505490291002100910A461D
:1056B0000B46019100F034F903B000BD3304000043
:1056C000410040020122400AD205090E80187F29BC
:1056D00001DA00207047962903DC9622511AC8404F
:1056E000704796398840704770B5CD0F4A0009035E
:1056F0000123090B1B0519430B4BED070024520D29
:105700009A4201DA002070BD074B34339A4203DC21
:105710009A1A00F093F802E00449511888402C438B
:10572000F1D0404270BD0000FF030000CDFBFFFF41
:105730004A0009030123090B1B051943094B10B546
:10574000520D9A4201DA002010BD064B34339A42C2
:1057500003DC9A1A00F072F810BD03495118884012
:1057600010BD0000FF030000CDFBFFFFC20FD207FA
:10577000400040080BD0C10D0723DB01C9184002CF
:105780000905400A1143C208400711437047002031
:105790000146704710B5002904DB0124E4074042AC
:1057A0008C412146002B04DB1C460123DB075242BF
:1057B000A341994200D1904210BD0000CB0FDB07FE
:1057C000490010B5490802460A4307D00A0D0724CC
:1057D0000903E401090B121B002A01DC002010BDA3
:1057E000C900440F0C43C100E018D205801800F036
:1057F00049F810BD0122D207002800DB101A002949
:1058000000DB511A814270470122D207002800DBD9
:10581000101A002900DB511A8842704710B5202A5F
:1058200004DB0146203A9140002010BD9140202326
:105830009C1A0346E3401943904010BD10B5202A3E
:1058400004DB0846203AD040002110BD0B46D3406F
:10585000D0402024A21A91400843194610BD10B52B
:10586000202A06DBCB170846203A1041C1170B430C
:1058700006E00B461341D0402024A21A9140084371
:10588000194610BD002904DA401C490001D1400826
:105890004000704770B40024050C05D110240004AA
:1058A00002D1002921D01124050E01D100020834B3
:1058B000050F01D10001241D850F01D18000A41C1A
:1058C000002801DB4000641C002908D020252E1B85
:1058D0000D46F540A14000D00121294308430106AF
:1058E0001B1B000ADB1D02D5002070BC7047DB05C6
:1058F000181880180029F8DA401C4900F5D170BC4E
:1059000040084000704710B5002B08DA0024401C06
:10591000614192185B411A4301D14008400010BD1B
:10592000F0B51FB482B005460C0003D0084605F060
:10593000D1FA02E005F0CEFA20300246009021466E
:105940002846FFF76BFF049B059A04460F46184351
:105950001143084314D0184610431BD0009840212F
:105960000A1A18460599FFF769FF05460E46009A80
:1059700005990498FFF752FF084305D0012004E081
:105980002046394607B0F0BD0020C11705430E433D
:105990002C43374300990E986305401A7905E40AB1
:1059A00000220C43FD0A0A3002D500200146E9E737
:1059B0000105101969410C9C0D9D00196941FFF703
:1059C000A2FFDFE7064C0125064E05E0E36807CCA1
:1059D0002B430C3C98471034B442F7D3FFF774FBC9
:1059E0003CC100085CC1000870B58C180578401CEB
:1059F0006B075B0F01D10378401C2A1106D1027896
:105A0000401C03E006780E70401C491C5B1EF9D157
:105A10002B0705D40023521E0DD40B70491CFAE746
:105A20000378401CCB1A921C03E01D780D70491CB2
:105A30005B1C521EF9D5A142D8D3002070BD0000D6
:105A400038B50446074908480068FFF751FB604332
:105A5000009002E00098401E009000980028F9D1C4
:105A600038BD000040420F008801002070B5044698
:105A70000025206880688007800F012807D12068F2
:105A80000068C007C00F002801D0012000E00020FE
:105A9000002839D1206880681C490840002801D1BD
:105AA000012000E00020002809D1606D102108438A
:105AB0006065A06D01210843A065012070BD2068CC
:105AC000806801210843216888600120FFF7B8FF42
:105AD00001F014FA05460EE001F010FA401B0A2806
:105AE00009D9606D102108436065A06D012108434C
:105AF000A0650120E2E720680068C007C00F01210F
:105B0000484048400028E7D00020D7E71700008031
:105B100010B502460B460020002103E0545C241817
:105B2000A0B2491C9942F9D3C443A0B210BD0000F1
:105B300010B5034800F0DCFE024800F0D9FE10BDAD
:105B4000DC1700209417002030B51C25446C2C4035
:105B50000125A540046C6560046863608468102CAE
:105B600004D10468A2600468E16003E00468A160F5
:105B70000468E26030BD000001201749487202202D
:105B80001649487203201649487204201549487284
:105B9000114815490A7842714978817110481249B3
:105BA0000A784271497881710C480F490A7842702D
:105BB000497881700B480C490A78427049788170A5
:105BC0000A4809490A7842704978817006490A787A
:105BD0004271497881717047BC1100201A1200206F
:105BE000DE110020D01100204401002030120020DE
:105BF00010B504F02BFA202004F0E0FA012005F0A3
:105C000085FD002004F0DAFA044805F0EDFB0448B5
:105C100005F01EFF002005F05BFF10BD61000020B5
:105C20008380000010B501210520000701F052F922
:105C3000002802D000200C49086002210B4801F026
:105C400049F9002809D108490860094800880A2153
:105C500048430849088005F021F8012001F034F894
:105C6000022001F031F810BD800100200004005036
:105C700060010020740100207047000000210A4AE2
:105C800051610A494968012252021143074A516091
:105C90001146496808221143044A51600021C20993
:105CA000D20111607047000024180020002002403B
:105CB0007FB504460D460020039000F0BDFF002094
:105CC00000900194E809029003A9684600F036FFAD
:105CD000002804D000F078FF002004B070BD00F070
:105CE00073FF0120F9E710B50346002002E01C5CB9
:105CF0000C54401C9042FAD310BD000000203949DA
:105D00008969FF2201321140914208D1364949691F
:105D100002221143344A5161FF21013108433149C4
:105D20008969012252021140914208D12E494969E4
:105D3000012211432C4A516101214902084329499A
:105D40008969012292021140914208D1264949698C
:105D500008221143244A5161012189020843214943
:105D600089690122D2021140914208D11E49496934
:105D7000042211431C4A51610121C90208431949F7
:105D80008969012252031140914208D1164949699B
:105D900010221143144A516101214903084311495A
:105DA0008969012252041140914207D10E49496983
:105DB000202211430C4A5161202108430949896975
:105DC000012212041140914208D107494969402239
:105DD0001143054A516101210904084301498861C1
:105DE00070470000002002402418002070B50446CF
:105DF00001F084F805460BE0601C002808D0002C58
:105E000004D001F07BF8401BA04201D9032070BDF3
:105E10001F488069C007C00F0028EDD11C48806969
:105E200002210840022801D1194988611848806977
:105E3000FF2101310840884223D01548806949007C
:105E4000084088421DD012488069490008408842B5
:105E500017D00F48806949000840884211D00C488B
:105E600080698900084088420BD00948806909018F
:105E70000840884205D00648806949100840884299
:105E800003D1FFF73BFF0120C1E70020BFE700007F
:105E900000200240F0B585B006460F4614460025A6
:105EA000029601970020009000F0C6FE13E00198D2
:105EB000006803900220039A029900F095FE00907A
:105EC0000098002800D008E00298001D0290019878
:105ED000001D01902D1DA542E9D300BF00F074FE06
:105EE000A54202D2002005B0F0BD0120FBE7000072
:105EF0000246002108E04800064B185A904201D1A2
:105F000008467047481CC1B2034800788142F2DB62
:105F100000BFF6E72A1400202801002070B50446CF
:105F20000D462946204600F0DEFF70BDFEB50C4848
:105F300001F0F2F980B202900298FFF7B3FB044639
:105F4000084A094BFFF7A8FA0022084B019100907C
:105F5000FFF70AFB0646FFF7EBFB80B2FEBD000031
:105F60008C160020F853E3A59B843E4000408F40F0
:105F700010B5454845490A784270497881704449CE
:105F80000A7842714978817105203F49487296200C
:105F900005F04CFD4B20C00005F064FD00223A499D
:105FA0000C2005F061FE00210C2005F071FE02209E
:105FB00005F096FD00BF00210F2005F08FFC35494C
:105FC0000860354908400028F5D032480068401C78
:105FD000002801D103F0A0F82E48006801218903B0
:105FE000084000283FD08122D20100210F2005F077
:105FF000F4FD0021102005F071FC4406640E2146DA
:106000000022264805F0BAFC2448407A05283AD1F7
:1060100002221F492148401DFFF7E8F8002832D12D
:106020001E48807A1E49087004221C49491C1D48DC
:10603000FFF7B8F81B48006800F042F81A490880DA
:1060400017480078420015490B311848FFF7AAF8A5
:1060500015480088164909884843164908800220D7
:10606000154908700FE0104908880988491E0E4B31
:10607000198012490988FFF751F80D4800884143FB
:1060800088B20C49088010BD3012002002010020A7
:10609000440100207000002000D02724801200203E
:1060A0002801002030010020FC0000202A140020DC
:1060B00056010020520100206000002058010020FD
:1060C00070B50646174801F027F9C5B22846E9170A
:1060D000C90E091849114901691ACCB209E03046C4
:1060E000E040C007C00F002801D1204670BD601CF1
:1060F000C4B20D4800888442F1DB012409E0304637
:10610000E040C007C00F002801D12046EEE7601C28
:10611000C4B2054800888442F1DB03480078401E81
:10612000C0B2E3E78C1600205801002010B50B48E0
:1061300000F074FB0A21094800F0FAFA074800F061
:10614000A1F9012149020840884204D1034800F026
:106150009CF980B210BD00BFFCE7000030160020A3
:10616000F0B587B000220121424800F0C0FEFFF7E1
:10617000DDFF0546FFF77BFA04463F49FFF79CF831
:106180003E490860012211463A4800F0B0FE3B4803
:106190000068FFF7EBFA04460022394BFFF7FAFAE2
:1061A0005ED838480078002821D000203549087092
:1061B000FFF7BCFF0546FFF75AFA04462E49FFF7E2
:1061C0007BF82E49086008460068FFF7CFFA0446BE
:1061D00000222B4BFFF752F900222B4B0591049024
:1061E000FFF75AF90646FFF7E9FA284908602348FD
:1061F0000068FFF7BBFA06460022214BFFF73EF985
:106200000446234A234BFFF747F9039102901F48A6
:106210000068FFF7ABFA04461D4A52421E4BFFF7D7
:106220003BF901910090039B029AFFF783F80591D7
:106230000490FFF7C3FA154908601849134800682D
:10624000FFF7E2FA02D215481049086000210F4812
:106250000068FFF7CFFA06D200200C49086002E080
:1062600000200A49086009480068FFF729FAC0B20F
:1062700007B0F0BD0004005000401B44280000207F
:1062800000000C403000002000E064402C000020A2
:106290003333333333B33040CCCCEC3F0000C8420F
:1062A000F8B5044600250026002700BF5020005DF9
:1062B000012801D10220F8BD01215020015500BF65
:1062C000206880688007800F012806D12068006858
:1062D0000840002801D0012000E00020002841D122
:1062E000606DFF2101318843022108436065206809
:1062F000C0688707BF0F2068C068800880002168D9
:10630000C860206880680121C90708432168886047
:1063100000F0F4FD064611E000F0F0FD801B0A28B5
:106320000CD9606D0221884310210843606500BFCD
:1063300000215020015500BF0120BCE72068806883
:10634000C00FC0070121C9078842E5D02068C06896
:1063500038432168C860606D0221884301210843E9
:10636000606504E0606D202108436065012500BF81
:1063700000215020015500BF28469CE770B5044617
:106380000D4600BF5020005D012801D1022070BDE4
:1063900001215020015500BF206880680421084079
:1063A000800800280AD0606D20210843606500BF86
:1063B00000215020015500BF0120E8E72D49686801
:1063C000884229D02068806A29684903490B08431C
:1063D0002168886228684003400B27490840012152
:1063E0008904884208D12548806849010843234927
:1063F00088600A20FFF724FB28684003400B2049EF
:1064000008400121490488422CD11C488068490178
:1064100008431A49886025E02068806A2968490392
:10642000490B88432168886228684003400B124961
:10643000084001218904884205D11048806849013B
:1064400088430E49886028684003400B0C49084087
:1064500001214904884205D10848806849018843E0
:106460000649886000BF00215020015500BF002070
:106470008DE70000011000000000044800270140E3
:10648000000002440146486D704701460868006CF0
:106490007047000010B50446002C01D1012010BD4A
:1064A000606D002806D1A0650021502001552046CE
:1064B00000F00EF9606D10210840102806D0206809
:1064C000806804210840800800280AD0606D1021EF
:1064D0000843606500BF00215020015500BF012026
:1064E000DDE7606DFF2101318843022108436065CB
:1064F000206880688007800F012807D12068006825
:10650000C007C00F002801D0012000E000200028B3
:106510003AD100BF032189076068884207D0494209
:106520006068884203D04900606888420CD12068C6
:10653000006980008008216808612068006961683E
:1065400008432168086112E0206800698000800823
:10655000216808615C4880680F21890488435A4992
:10656000886008468068616808435749886000BFB2
:106570002068C068182188432168C8602068C06806
:10658000A16808432168C8604F4880680121490616
:1065900088434D49886008468068A18E49060843B3
:1065A000494988602068806801210907084000285F
:1065B00004D1206880680843216888602068C0682A
:1065C000424908402168C8602169E068022901D178
:1065D000042100E0002108432021095D490308430C
:1065E0002C21095D49000843216B0843A1698903F7
:1065F0000843E169C90308432168C9680843216861
:10660000C860FF21C231606A884207D0A16A606A0F
:1066100008432168C96808432168C8602120005DDB
:10662000012813D12020005D002807D12068C06810
:106630000121090408432168C86007E0606D20213A
:1066400008436065A06D01210843A065E06B012847
:1066500017D120680069FF218900884321680861FB
:10666000216C606C0843A16C0843216809690843E8
:1066700021680861206800690121084321680861D8
:106680000BE020680069C007C00F002805D0206813
:106690000069400840002168086120684069C0081E
:1066A000C0002168486120684069A16B08432168E7
:1066B00048610020A065606D0221884301210843E4
:1066C00060650020EBE60000002701401902FEFF94
:1066D00010B586B00446142101A8FEF77CFD1249CE
:1066E000206888421ED11148406B491508430F4964
:1066F000486300BF0846C06A012108430B49C862CD
:106700000846C06AC007C00F009000BF00BF02204B
:106710000190032002900020039001A905200007AA
:1067200000F0E2FA06B010BD002401400010024063
:10673000F8B504460D46002600276069082801D1F7
:10674000082711E02068C068C007C00F00280AD0E1
:10675000606D20210843606500BF00215020015575
:1067600000BF0120F8BD0C2700F0C8FB064614E06E
:10677000681C002811D0002D04D000F0BFFB801B46
:10678000A8420AD9606D04210843606500BF00215A
:106790005020015500BF0320E4E72068006838401E
:1067A0000028E5D0606D012149020843606520683A
:1067B000C068032189020840002826D12020005DFE
:1067C000002822D1206800680821084008281CD130
:1067D0002068806804210840800800280DD12068C6
:1067E00040680C21884321684860606DFF210131B9
:1067F000884301210843606507E0606D202108435C
:106800006065A06D01210843A065A069002802D140
:106810000C20216808600020A4E7000070B5044641
:1068200000252068806804210840800800282BD1BA
:1068300000BF5020005D012801D1022070BD012160
:106840005020015500BFE069012803D02046FFF722
:106850000DF90546002D18D1606D0D490840FF2146
:106860000131084360650020A06500BF0021502071
:10687000015500BF1C202168086020688068042141
:1068800008432168886000E002252846D6E700001A
:10689000FEF1FFFF70B5044600252520005D0228AB
:1068A00003D00420E063012520E0206800680E2169
:1068B000884321680860206800684008400021681B
:1068C00008601C21606C084001218140206C4160FF
:1068D00001212520015500BF00212420015500BFC2
:1068E000A06B002802D02046A16B8847284670BDC7
:1068F00070B50446206C0568206806681C20616C31
:10690000014004208840284000281DD00420304049
:10691000002819D02068006820210840002805D1EF
:106920002068006804218843216808601C21606C8D
:10693000084004218140206C4160206B00285AD01F
:106940002046216B884756E01C20616C01400220E4
:1069500088402840002825D002203040002821D03F
:106960002068006820210840002808D120680068BD
:106970000A218843216808600121252001551C2136
:10698000606C084002218140206C416000BF002102
:106990002420015500BFE06A00282CD02046E16A7F
:1069A000884728E01C20616C01400820884028406E
:1069B000002820D00820304000281CD02068006823
:1069C0000E218843216808601C21606C0840012169
:1069D0008140206C41600120E063012125200155A8
:1069E00000BF00212420015500BF606B002802D0A9
:1069F0002046616B884770BD70B50446002C01D1FC
:106A0000012070BD244A2168881A1421FEF770FB0A
:106A10008000606420480838206402212520015548
:106A2000206805681D480540E168A06808432169A1
:106A3000084361690843A1690843E1690843216A81
:106A4000084305432068056001218903A068884246
:106A500017D011487830806A1C22616C11400F22D7
:106A60008A4090430C49783188621C22616C114045
:106A70006068884008497831896A08430649783156
:106A800088620020E0630121252001550021242097
:106A900001550020B5E70000080002400F80FFFF0D
:106AA000F8B504460D4616461F460020009000BF6C
:106AB0002420005D012801D10220F8BD01212420FD
:106AC000015500BF2520005D01282DD10221252080
:106AD00001550020E06320680068400840002168FC
:106AE00008603B46324629462046FFF72DF8206BCA
:106AF000002806D0206800680E210843216808603D
:106B00000BE0206800680421884321680860206841
:106B100000680A2108432168086020680068012194
:106B200008432168086006E000BF002124200155C9
:106B300000BF022000900098BFE70000F8B50446AF
:106B40000E460127002500BF1C48007C012801D10A
:106B50000220F8BD01201949087400BF1848FFF74A
:106B600045F90746002F22D1401E3060656817E0C6
:106B70002846FFF783F81248FFF738F9074611480F
:106B80004068082188430F49486008464068491515
:106B900088430C494860002F01D0356006E08035FD
:106BA000A068C00161684018A842E1D800BF00BFDA
:106BB00000200249087400BF3846CAE724180020A4
:106BC00050C30000002002400648406802210843EC
:106BD000044948600846406801210843014948606B
:106BE0000020704700200240F8B507460C461546C5
:106BF000012600BF0E48007C012801D10220F8BD0B
:106C000001200B49087400BF0A48FFF7EFF8064659
:106C1000002E06D10649486125600648FFF7E6F8D0
:106C2000064600BF00200249087400BF3046E6E770
:106C30002418002050C300001D484068C007C00F42
:106C4000002816D000BFEFF31080014600BF72B6D7
:106C50001848174AD0601848D06000BF81F31088E8
:106C600000BF10464068C007C00F002801D00120B7
:106C700070470F48406802221040022815D100BF1B
:106C8000EFF31080014672B60C48094A10610C48B7
:106C90001061084680F3108800BF10464068022249
:106CA0001040022801D10120E2E70020E0E70000C7
:106CB00000200240EFCDAB8905040302BFAE9D8CDE
:106CC000161514137047000010B5044605484069B6
:106CD0002040002804D0034844612046FFF7F2FF1B
:106CE00010BD00000004014070B5034600220024DE
:106CF0000020DAE0012696400D6835402C46002C35
:106D000077D04D68022D02D04D68122D15D1D508CF
:106D1000AE001D462035A8595507EE0E0F25B5408B
:106D20000646AE4330465607F60E0D69B540284379
:106D3000D508AD001E46203670514D68012D08D093
:106D40004D68022D05D04D68112D02D04D68122DD1
:106D500018D1986856000325B5400646AE43304624
:106D60005600CD68B5402843986058680125954085
:106D70000646AE43304610264D6835402D099540F5
:106D800028435860186856000325B5400646AE43B0
:106D900030460D79AD07AD0F5600B5402843186059
:106DA000D86856000325B5400646AE433046560027
:106DB0008D68B5402843D860012636074D683540B8
:106DC000B54271D13C4D6D6B012635433A4E75632A
:106DD0003A4D9608B600A85995072E0F0F25B540D5
:106DE0000646AE43304605252D07AB4202D10025AD
:106DF00015E059E0324DAB4201D101250FE0314D94
:106E0000AB4201D102250AE02F4DAB4201D103254F
:106E100005E02E4DAB4201D1052500E00625960781
:106E2000360FB5402843254D9608B600A851284D89
:106E300028680546A5432846012636044D68354096
:106E4000B54202D1054625432846214D2860686891
:106E50000546A5432846012676044D683540B542CF
:106E600002D1054625432846194D6860A8680546A5
:106E7000A5432846012636054D683540B54202D166
:106E8000054625432846124DA860E8680546A543F7
:106E90002846012676054D683540B54202D10546A3
:106EA000254328460A4DE860521C0D68D540002D48
:106EB00000D01FE770BD0000001002400800014034
:106EC0000004005000080050000C0050001C00504E
:106ED00000040140024613690B40002B01D0012041
:106EE00000E00020704742694A4042617047002A32
:106EF00001D0816100E081627047000001480068B4
:106F0000704700008401002002480068401C0149CD
:106F1000086070478401002010B50024084800680C
:106F20004021084306490860002000F00BF80028C3
:106F300001D0012401E000F025FA204610BD000038
:106F40000020024070B5044600257D21C900094893
:106F50000068FEF7CDF8064601F0D4F8002801D00D
:106F6000012504E000222146501E00F033FA284695
:106F700070BD0000880100207047704770B505465D
:106F80003C480078401C3B49087001203A49087091
:106F90003A480088401C394908803948008803F085
:106FA000C5F83849C888FEF762FB06463649FEF741
:106FB00083F90446354801682046FEF724F9334931
:106FC000086002213248FFF785FF002819D12D49BA
:106FD000C888FEF74CFB06462B49FEF76DF90446C0
:106FE0002C4801682046FEF70EF92A4908602A4914
:106FF00028480068FEF708FC06D828482849C860D9
:1070000002E0002023490860264920480068FEF776
:10701000FBFB03D201202449087002E00020224932
:1070200008701849498F481EFEF716FB044617489A
:1070300001682046FEF7DEFB09D81C4800780028CE
:1070400005D01B48C079012108431949C8710D4971
:10705000488FFEF70CFB04460C4801682046FEF7FB
:10706000C9FB05D211480078002801D004F014FFB4
:1070700070BD00007E010020510100206C01002045
:1070800052010020BC0D002000007A448001002045
:1070900000040050780100200000A0400400FA0520
:1070A00000ED00E0000040402E01002066010020BD
:1070B00030120020704710B50446002C01D1012089
:1070C00010BD02212E200155204601F077FD2046FB
:1070D00000F0F4F800212E20015500BF2D200155AD
:1070E00000BF0020ECE77047704710B504462068E9
:1070F0000068C007C00F01214840484000280CD05C
:1071000020688068084048404840002805D0012099
:10711000216848602046FFF731FF2068006802219F
:107120000840400800280BD02068806808404008CC
:10713000002805D00220216848602046FFF71CFF88
:107140002068006804210840800800280BD02068CF
:10715000806808408008002805D004202168486025
:10716000204600F00DF92068006808210840C0089A
:1071700000280BD0206880680840C008002805D08F
:107180000820216848602046FFF794FF20680068C7
:1071900010210840000900280BD0206880680840B2
:1071A0000009002805D01020216848602046FFF71C
:1071B000E4FE2068006820210840400900280BD028
:1071C0002068806808404009002805D020202168F8
:1071D00048602046FFF788FF20680068402108408B
:1071E000800900280BD020688068084080090028AA
:1071F00005D04020216848602046FFF774FF10BD8D
:1072000070B50446002C01D1012070BD60680128D2
:1072100000D100BF26496069884200D000BF2E20FF
:10722000005D002805D100212D200155204600F0E9
:1072300059F802212E2001552068C5686068012890
:1072400003D08905A06A884203D11E2128468843BD
:10725000054617496069884201D01648054016481E
:107260000540A16860680843216A0843616A0843D1
:10727000A16A084305436068012804D00121C905BB
:10728000A06A884203D1E1682069084305430849A0
:107290006069884205D06169A0690843E1690843D3
:1072A00005432068C56001212E2001550020ACE770
:1072B000FFFF00003F1FFFFFF8F119FF10B5044664
:1072C00006492068884208D10548806B4000400884
:1072D000034988630D2000F065F810BD007C004074
:1072E0000010024010B504460949206888420DD1BB
:1072F0000848806B4905084306498863002201213C
:107300000D2000F067F80D2000F058F810BD0000C7
:10731000007C00400010024001460868C0697047C8
:1073200010B5034602242E20C454144800682407D4
:107330002043124C20601868C0680124E4042043F4
:107340001C68E06018688068012420431C68A06005
:1073500018680069012420431C6820611868816155
:107360001868426118680069042420431C68206181
:1073700001242E20C454002010BD00000004014050
:10738000704700000648406B0121084304494863E8
:107390000846806B09040843014988637047000070
:1073A0000010024000BFC206D20E01219140024AE5
:1073B000116000BF7047000080E100E000BFC2061E
:1073C000D20E01219140024A116000BF70470000B7
:1073D00000E100E070B504460D46164629462046F9
:1073E00001F05EFE70BD0000024949688143014A18
:1073F000516070470070004003480068FF21013170
:10740000084301490860704700700040024949681C
:107410000143014A5160704700700040074800680E
:107420000221084305490860054800690421084312
:107430000349086100BF00BF30BF704700700040C3
:1074400000ED00E010B5024600200E4B18688008E1
:1074500080000346134318460A4B18600A4B1B6909
:1074600004242343084C2361012901D130BF02E0E9
:1074700040BF20BF20BF044B1B690424A343024C20
:10748000236110BD0070004000ED00E0F8B5044637
:1074900020212068084020287CD12068084020282E
:1074A00000D100BF00278148806B012109070840F7
:1074B000002805D17D48806B08437C4988630127FB
:1074C0007B480068FF2101310840002816D1784828
:1074D0000068084376490860FFF710FD064606E09D
:1074E000FFF70CFD801B642801D90320F8BD70480C
:1074F0000068FF21013108400028F1D06B48056881
:10750000032109050D4060680840A8420DD009110B
:1075100060680840884208D1644800680121490435
:107520000840884201D10120E0E76048403000690E
:107530000321090408400546002D3DD0606808403D
:10754000A84239D0202120680840202834D157484B
:107550004030006903210904884305465348403000
:1075600000690121C90408435049403108610846B7
:1075700000690121C90488434C494031086108462B
:107580000561801528408915884215D1FFF7B6FCA2
:10759000064608E039E0FFF7B1FC801B4549884208
:1075A00001D90320A2E74148403000690121490286
:1075B0000840400A0028EED000BF00BF03210904A4
:1075C0006068084088420AD1384800680901884349
:1075D000032212056168114008433449086000BF66
:1075E00032484030006903221204616811400843A8
:1075F0002E494031086100BF012F05D12B48806B17
:10760000890588432949886300BF2078C007C00FD7
:10761000002809D025484030C06880088000A16853
:10762000084322494031C8600221206808400228EE
:1076300009D11E484030C0680C218843E1680843E6
:107640001A494031C86004212068084004280AD142
:1076500016484030C06803218902884321690843E5
:1076600012494031C86008212068084008280AD122
:107670000E484030C068032109038843616908430C
:107680000A494031C86080212068084080280AD11A
:1076900006484030C068032189048843A169084333
:1076A00002494031C860002020E70000001002407D
:1076B0000070004088130000F8B504460D46002C09
:1076C00001D10120F8BD79480068C007C00FA84269
:1076D0000ED276480068400840002843734908608D
:1076E00008460068C007C00FA84201D00120E9E7A2
:1076F000022120680840022807D16D48C068F021A7
:107700008843A16808436A49C8602078C007C00F51
:1077100000284CD06068022809D165480068012122
:1077200049040840400C002824D10120CAE76068C1
:10773000032809D15E480068012149060840400E2F
:10774000002817D10120BDE76068012808D15848FA
:10775000006804210840800800280BD10120B1E70F
:1077600053480068012149020840400A002801D11D
:107770000120A7E74E48C068800880006168084380
:107780004B49C860FFF7BAFB0646606802280FD174
:1077900007E0FFF7B3FB801B4649884201D903206D
:1077A00090E74348C0680C2108400828F1D134E034
:1077B000606803280FD107E0FFF7A0FB801B3D495D
:1077C000884201D903207DE73948C0680C21084070
:1077D0000C28F1D121E0606801280FD107E0FFF704
:1077E0008DFB801B3349884201D903206AE730486A
:1077F000C0680C2108400428F1D10EE007E0FFF733
:107800007DFB801B2B49884201D903205AE7284879
:10781000C0680C2108400028F1D124480068C00746
:10782000C00FA8420ED921480068400840002843F4
:107830001E49086008460068C007C00FA84201D072
:1078400001203FE7042120680840042808D1184897
:10785000C068072109028843E16808431449C860E9
:10786000082120680840082809D11148C06807216C
:10787000C90288432169C90008430D49C86000F066
:1078800049F80B49C968F022114009090A4A515CBC
:10789000C8400A4908600020FFF754FB0746002F44
:1078A00001D038460EE700200CE70000002002401F
:1078B00000100240881300001AC10008880100204F
:1078C00001480068704700008801002000B5FFF7FC
:1078D000F7FF0549C968072212021140090A034A45
:1078E000515CC84000BD0000001002402AC10008E1
:1078F00000B5FFF7E5FF0549C9680722D20211402C
:10790000C90A034A515CC84000BD00000010024093
:107910002AC10008FEB52E48C7680C203840002850
:1079200045D0042804D008280CD00C283ED10BE008
:107930002748006810210840002801D0254C00E0AD
:10794000254C41E0254C3FE00F2080043840800C5E
:1079500023490E5C032080053840800D401C0190B7
:107960001B48C068012109040840002807D01B49B2
:10797000714308460199FDF7BBFB054614E0144826
:10798000006810210840002807D0124971430846BA
:107990000199FDF7ADFB054606E00F497143084626
:1079A0000199FDF7A5FB05462C460DE000BF0848F0
:1079B0004068072149030840400B00900098401C94
:1079C00001218140CC0300BF00BF2046FEBD000066
:1079D0000010024000093D000024F40000127A006B
:1079E00032C10008FEB50446002C01D10120FEBDC5
:1079F000F848C6680C210E40C768012109040F40F1
:107A00002078C007C00F002872D0082E04D00C2E9A
:107A10000FD1084687420CD1EE4800680121490485
:107A20000840400C002863D06068002860D1012025
:107A3000DDE700BF012109046068884205D1E548FF
:107A400000680843E349086027E0052109046068ED
:107A500088420ED1DF480068012189040843DD49CE
:107A6000086008460068012109040843D9490860F4
:107A700013E0D8480068012109048843D54908600B
:107A800008460068012109040840009000BFD14861
:107A9000006889008843CF49086000BF60680028FB
:107AA00013D0FFF72BFA054606E0FFF727FA401B35
:107AB000642801D903209AE7C648006801214904D7
:107AC0000840400C0028F0D012E0FFF717FA0546F6
:107AD00006E0FFF713FA401B642801D9032086E76C
:107AE000BC480068012149040840400C0028F0D13E
:107AF00002212068084002287AD1E0680290042E12
:107B000003D00C2E34D1002F32D1B24800680421AA
:107B100008408008002804D00298002801D10120E4
:107B200065E7AC4840681F210902884321690902C2
:107B30000843A8494860084600680921884302991B
:107B40000843A4490860FFF7E5FEA249C968F0228E
:107B500011400909A04A515CC840A04908600020B2
:107B6000FFF7F0F901900198002841D001983EE715
:107B70000298002824D09748006809218843029978
:107B8000084394490860FFF7B9F9054606E0FFF796
:107B9000B5F9401B022801D9032028E78D48006869
:107BA0000421084080080028F1D08A4840681F213D
:107BB000090288432169090208438649486017E0A1
:107BC000844800684008400082490860FFF796F941
:107BD000054606E0FFF792F9401B022801D9032071
:107BE00005E77C4800680421084080080028F1D19E
:107BF000102120680840102867D1002E36D1754822
:107C0000006849010840400A002804D0A069002803
:107C100001D10120EBE66F48406807214903884302
:107C2000216A08436B494860084640680002000A20
:107C3000217F0906084367494860206A400B401CC1
:107C400001218140C8036349C968F0221140090934
:107C5000614A515CC840614908600020FFF772F931
:107C60000190019800284BD00198C0E6A069002837
:107C70002CD058480068FF2101310843554908605D
:107C8000FFF73CF9054606E0FFF738F9401B0228EC
:107C900001D90320ABE64F480068012149020840A2
:107CA000400A0028F0D04B48406807214903884328
:107CB000216A084347494860084640680002000AB4
:107CC000217F090608434349486019E0414800689C
:107CD000FF21013188433F490860FFF70FF905464E
:107CE00006E0FFF70BF9401B022801D903207EE6CE
:107CF00038480068012149020840400A0028F0D1B4
:107D0000082120680840082839D1606900281BD064
:107D1000304840300069012108432E494031086154
:107D2000FFF7ECF8054606E0FFF7E8F8401B0228ED
:107D300001D903205BE62748403000690221084052
:107D400040080028F0D01AE022484030006940087E
:107D50004000204940310861FFF7D0F8054606E0B1
:107D6000FFF7CCF8401B022801D903203FE6194851
:107D7000403000690221084040080028F0D1042169
:107D800020680840042879D1002000901148806BB9
:107D900089060840002806D10E48806B08430D492B
:107DA0008863012000900E480068FF2101310840DF
:107DB00000281ED10A480068084309490860FFF7F7
:107DC0009DF805460EE0FFF799F8401B642809D995
:107DD00003200CE6001002401AC1000888010020B0
:107DE0000070004085480068FF21013108400028EC
:107DF000E9D000BFFF210131A068884205D1804849
:107E0000006908437E49086130E0A06800280DD170
:107E10007B480069FF2101318843794908610846A0
:107E2000006909158843764908611FE005210902A8
:107E3000A06888420DD17248006901218902084377
:107E40006F49086108460069891508436C49086153
:107E50000CE06B480069FF210131884368490861E3
:107E600008460069091588436549086100BFA06894
:107E7000002815D0FFF742F8054608E031E0FFF78B
:107E80003DF8401B5F49884201D90320AFE55C48BB
:107E90000069012149020840400A0028EFD013E0A0
:107EA000FFF72CF8054607E0FFF728F8401B554977
:107EB000884201D903209AE551480069012149020D
:107EC0000840400A0028EFD10098012808D14C480A
:107ED0004038806B0121090788434949403988634C
:107EE00000BF606A00284CD00C2E69D0606A02285E
:107EF00048D1434840380068012109068843404979
:107F000040390860FEF7FAFF054606E0FEF7F6FF87
:107F1000401B022801D9032069E539484038006830
:107F2000012149060840400E0028EFD1E16AA06A0D
:107F30000843216B084332494039C968FD221204C5
:107F4000914308432E494039C86008460068012122
:107F5000090608432A4940390860FEF7CFFF054665
:107F600006E0FEF7CBFF401B022801D903203EE5C7
:107F7000234840380068012149060840400E002887
:107F8000EFD038E01E4840380068012109068843D8
:107F90001B4940390860FEF7B1FF054606E0FEF7D1
:107FA000ADFF401B022801D9032020E514484038CA
:107FB0000068012149060840400E0028EFD11AE070
:107FC000606A012800D112E50D484038C7680120D9
:107FD00000043840A16A88420BD10F208004384049
:107FE000E16A884205D1032080053840216B884230
:107FF00001D00120FBE40020F9E400000070004003
:10800000401002408813000010B50446002C01D136
:10801000012010BD606A002800D100BF0021A162CC
:108020005120005D002804D150200155204600F069
:1080300035F802215120015520680068402188430D
:1080400021680860A16860680843E1680843216905
:1080500008436169084301225202A16911400843A3
:10806000E1690843216A0843A16A0843216808605E
:10807000A069000C04210840616A08432168486037
:108080002068C069910088432168C861002060654C
:108090000121512001550020BBE7000010B586B03A
:1080A0000446142101A8FDF796F814492068884277
:1080B00022D11348406B891408431149486300BF1B
:1080C0000846C06A012108430D49C8620846C06AD3
:1080D000C007C00F009000BF00BFE0200190022049
:1080E000029000200390032004900020059001A935
:1080F00005200007FEF7F8FD06B010BD0030014076
:108100000010024070B504462546681E09498842A1
:1081100001D901200CE0681E074948610321081FAE
:1081200000F0BEFF0020044988610720086100209C
:1081300070BD0000FFFFFF0000E000E070477047E7
:10814000FEB504462068C56920680668206887680F
:108150002807000F0190019800280ED12020284008
:1081600000280AD020203040002806D0206E0028A9
:1081700002D02046216E8847FEBD019800287DD0A0
:10818000F807C00F002804D1FF202130304000281C
:10819000F5D0E807C00F00280BD0FF200130304099
:1081A000002806D0012021680862E06F0121084301
:1081B000E0670220284000280AD0F807C00F0028F6
:1081C00006D0022021680862E06F04210843E067BE
:1081D0000420284000280AD0F807C00F002806D045
:1081E000042021680862E06F02210843E06708204C
:1081F000284000280ED020203040002803D1F80766
:10820000C00F002806D0082021680862E06F08210E
:108210000843E067E06F002846D02020284000286F
:1082200009D020203040002805D0206E002802D040
:108230002046216E8847E06F0090206880684021CA
:108240000840402804D0082100980840002826D083
:10825000204602F074FA20688068402108404028D7
:1082600019D120688068884321688860E06E002802
:108270000DD02548E16E8863E06E00E015E0FEF762
:1082800009FB002810D0E06E816B88470CE0204687
:10829000FFF755FF08E02046FFF751FF04E02046B6
:1082A000FFF74DFF0020E06766E70120000528404A
:1082B00000280CD0012080053840002807D001207C
:1082C0000005216808622046FFF738FF54E7802048
:1082D000284000280AD080203040002806D0606E58
:1082E000002802D02046616E884745E7402028409C
:1082F000002807D040203040002803D0204602F05C
:1083000030FA39E700BF37E77DA6000810B504460C
:10831000002C01D1012010BDA069002800D000E090
:1083200000BF606F002805D1002170200155204654
:1083300000F02CF8242060672068006840084000A6
:1083400021680860204602F073FA012800D1E2E7B4
:10835000606A002802D0204602F002F820684068D7
:108360000921C902884321684860206880682A2161
:1083700088432168886020680068012108432168DB
:108380000860204602F064F8C5E7000010B586B02A
:108390000446142101A8FCF71EFF364920688842D4
:1083A00066D13548406B012189030843324948634F
:1083B00000BF0846C06A012108432F49C862084629
:1083C000C06AC007C00F009000BF00BF032040027A
:1083D00001900220029000200390032004900420CA
:1083E000059001A905200007FEF77EFC23482449DB
:1083F000086003204860002121488160C16080211D
:1084000001610021416181612021C1610902016294
:10841000FEF7F2FA002801D0FDF72EFC00BF184845
:10842000E066846200BF15481438164908600320CE
:1084300048601021134881600021C16080210161E2
:10844000002141618161C1610162FEF7D5FA002816
:1084500001D0FDF711FC00BF0A48A066846200BF8E
:10846000002201211B20FEF7B5FF1B20FEF7A6FF0F
:1084700006B010BD0038014000100240300002403C
:1084800094170020DC17002070B504460D461646F0
:10849000A06F202863D1002D01D0002E01D1012032
:1084A00070BD01210903A068884208D12069002815
:1084B00005D1E807C00F002801D00120F0E700BF78
:1084C0007020005D012801D10220E9E70121702020
:1084D000015500BF6565582006530020E067222043
:1084E000A067E06E002820D01E48E16EC8621E48DA
:1084F000E16E08631D48E16E48630020E16E886309
:108500002368194624313346626DE06EFEF7C8FADF
:1085100000280AD01020E06700BF0021702001551C
:1085200000BF202060670120BAE700BF0021702053
:10853000015500BF20680068FF2101310843216810
:1085400008602068806801210843216888602068ED
:10855000806840210843216888600020A0E702204D
:108560009EE70000E7A6000831A7000895A60008CE
:1085700070477047FFB583B004460D461746606FDD
:10858000202875D1002D01D0002F02D1012007B085
:10859000F0BD01210903A068884208D120690028A4
:1085A00005D1E807C00F002801D00120EFE700BF88
:1085B0007020005D012801D10220E8E70121702030
:1085C000015500BF0020E06721206067FEF796FCA0
:1085D0000190502007535220075301210903A0683E
:1085E000884205D12069002802D10026029502E0C8
:1085F0002E460020029021E0069800900022802163
:108600002046019B02F002FB002801D00320BEE7B8
:10861000002E09D102980088C005C00D216888622B
:108620000298801C029003E0307821688862761CF2
:108630005220005B401E81B2522001535220005B49
:108640000028D9D106980090002240212046019BA5
:1086500002F0DCFA002801D0032098E720206067B0
:1086600000BF00217020015500BF00208FE7FFE709
:1086700002208CE7704700BFFEE710B500220421FE
:1086800005200007FEF733FC002208210520000723
:10869000FEF72DFC0A2002F05FFE012204210520D6
:1086A0000007FEF724FC0A2002F056FE00220421F7
:1086B00005200007FEF71BFC10BD10B500220421A9
:1086C00005200007FEF713FC012208210520000702
:1086D000FEF70DFC0A2002F03FFE012204210520D6
:1086E0000007FEF704FC0A2002F036FE00220421F7
:1086F00005200007FEF7FBFB10BD70B50546002402
:1087000000261EE00022042105200007FEF7EFFBF3
:108710000A2002F021FE0122042105200007FEF7B5
:10872000E6FB6006040E082105200007FEF7D2FBD9
:10873000002801D0601CC4B2052002F00DFE701CA0
:10874000C6B2082EDEDB002D02D1FFF7B6FF01E036
:10875000FFF793FF204670BD70B504460022042148
:1087600005200007FEF7C3FB00252AE080202040FB
:10877000C011002806D00122082105200007FEF7BD
:10878000B6FB05E00022082105200007FEF7AFFB3D
:108790006006040E0A2002F0DFFD012204210520FC
:1087A0000007FEF7A4FB0A2002F0D6FD00220421F8
:1087B00005200007FEF79BFB0A2002F0CDFD681C98
:1087C000C5B2082DD2DB70BD10B5012208210520ED
:1087D0000007FEF78CFB0122042105200007FEF7AD
:1087E00086FB0022082105200007FEF780FB0A20F7
:1087F00002F0B2FD0022042105200007FEF777FBFE
:1088000010BD10B50022042105200007FEF76FFB04
:108810000022082105200007FEF769FB0A2002F06C
:108820009BFD0122042105200007FEF760FB0122C9
:10883000082105200007FEF75AFB0A2002F08CFDF4
:1088400010BD10B500240122082105200007FEF705
:108850004EFB062002F080FD0122042105200007C6
:10886000FEF745FB062002F077FD07E0601CC4B26E
:10887000FA2C03DDFFF7C5FF012010BD08210520FC
:108880000007FEF727FB0028F0D100220421052075
:108890000007FEF72CFB0020EFE7000038B501F0E1
:1088A0000FFE01F061FE6E480068C06902210840B9
:1088B000002802D06B486C49C860FDF737FB0446BE
:1088C0006A484088002808DD68484088401E81B218
:1088D0006648418001206649087065480078002894
:1088E00006D001280AD0022817D0032822D11BE085
:1088F000012291025F48FEF7FAFA1BE0212C06DA0A
:108900000022012189025B48FEF7F1FA04E001220E
:1089100091025848FEF7EBFA0CE00022012189028F
:108920005448FEF7E4FA05E0012291025148FEF7AF
:10893000DEFA00BF00BF0121C9024E48FEF7CAFAA5
:10894000002828D000204C4908604C4800780028B6
:1089500004D101204949087002F0A0F94848007884
:1089600063280BDD002208214248FEF7C0FA0122ED
:10897000D10305200007FEF7BAFA1BE00122082107
:108980003C48FEF7B4FA00220121C9030520000784
:10899000FEF7ADFA0EE000203849087000220821E9
:1089A0003448FEF7A4FA00220121C903052000077C
:1089B000FEF79DFA2D48808C012820D100253148F2
:1089C000009072B680213048FDF772F90546002DFF
:1089D00005D0022269462C48FDF75CFA054662B6CE
:1089E0002AA002F067FA00212048818403F004FBEA
:1089F000642002F0A7FC1B481B49C86000BF1B484D
:108A0000408C01280ED100211848418400201749CC
:108A10004039088003F0F0FA642002F093FC11481A
:108A20001149C8601148008C01280AD100210F4863
:108A3000018403F0E1FA642002F084FC09480A4949
:108A4000C8600A48403800881449884204D1074861
:108A50004038C088002802D102480349C86038BDA8
:108A6000141700200400FA0500ED00E0FC0D0020C2
:108A70003601002000040050800100206801002021
:108A800050010020AAAA0000384A0008BDF8C8EB2F
:108A9000C9FDBCB6C4A3CABD0D0A0000AA5500009A
:108AA00008B53721202000F077F80321212000F0BD
:108AB00073F84021222000F06FF80821232000F0F5
:108AC0006BF8AA21302000F067F802200B490887D4
:108AD0000846008FC1B2322000F05EF80121332039
:108AE00000F05AF85F21202000F056F8684600F0A8
:108AF00007F80A2002F030FC08BD0000BC0D002081
:108B000010B5044621460F2000F023F8002800D1BC
:108B100010BD0120FCE770B504460025FFF754FEA8
:108B20003220FFF719FEFFF78CFEE0B2FFF714FECC
:108B3000FFF787FEFFF748FE3320FFF70DFEFFF734
:108B400080FE0020FFF7D9FD0546FFF75AFE2846B4
:108B500070BD70B505460C462846FFF7DCFF207057
:108B6000012070BD70B504460D46FFF72DFE322082
:108B7000FFF7F2FDFFF765FEE0B2FFF7EDFDFFF74F
:108B800060FE2846FFF7E8FDFFF75BFEFFF739FEC2
:108B90000A2002F0E1FB70BD70B504460D4629467F
:108BA0002046FFF7DFFF012070BD000010B502482E
:108BB000FEF79BFA10BD00008C160020F0B585B0C2
:108BC00004460020039072B64F49206840180028E0
:108BD00006D14E48C068032189040840039000E094
:108BE00000BF00BF2068806802902068C0680190C4
:108BF0002068456920688669434920684018002834
:108C00000DD142484038806A490508433F49403900
:108C100088620846806A40004008886200E000BF21
:108C200000BF002D01D1002E5FD0374920684018C9
:108C3000002807D13548C068032189048843334997
:108C4000C86000E000BF00BF002D1DD02068006993
:108C5000012108432168086120684561FEF74EF94B
:108C6000074600BFFEF74AF9C01B00902068006865
:108C700008210840082804D07D21C90000988842B6
:108C8000F0D9082021684860002E1DD020680069B6
:108C9000012108432168086120688661FEF72EF9EA
:108CA000074600BFFEF72AF9C01B00902068006845
:108CB00010210840102804D07D21C9000098884266
:108CC000F0D91020216848600F492068401800281A
:108CD00009D10E48C06803218904884303990843D9
:108CE0000A49C86000E000BF00BF20680069400872
:108CF0004000216808610298216888600198216815
:108D0000C86062B605B0F0BD0084FFBF40100240ED
:108D10001CB50020009001901E481F4908600021EA
:108D20001D48C163012080071B49486000211A4883
:108D3000816007218163012101610021C160001D63
:108D400001774177001F8162FF21C231416200211A
:108D500024300172042124384161002101638161C2
:108D60004163C161FDF796FB002801D0FCF784FF49
:108D70000A4800908013019069460748FDF7FEFA03
:108D8000002801D0FCF778FF00210348FDF788FA9E
:108D90001CBD000000240140301600200200000429
:108DA00008B500BF0A48006B012108430849086361
:108DB0000846006BC007C00F009000BF00BF002234
:108DC00001210A20FEF706FB0A20FEF7F7FA08BD8C
:108DD0000010024000B587B0142102A8FCF7FBF98F
:108DE00000BF6548C06A042108436349C862084659
:108DF000C06A04210840019000BF00BF00BF5E4868
:108E0000C06A802108435C49C8620846C06A802164
:108E10000840019000BF00BF00BF5748C06A012151
:108E200008435549C8620846C06AC007C00F019090
:108E300000BF00BF00BF0846C06A022108434E4978
:108E4000C8620846C06A02210840019000BF00BF06
:108E500001221C2105200007FEF749F8012247499D
:108E60004748FEF744F8002246494548FEF73FF8D8
:108E700000229121090205200007FEF738F80120A1
:108E80000290414803900020049002A905200007A9
:108E9000FDF72AFF02200290032003900020049097
:108EA00002A905200007FDF71FFF0C2002901120EA
:108EB0000390002004900320059002A905200007DC
:108EC000FDF712FF10200290012003900020049073
:108ED0000220059002A905200007FDF705FF0120EB
:108EE00002901120039000200490059002A92448CC
:108EF000FDF7FAFE0220029024480390012004901E
:108F000002A91F48FDF7F0FE2148029001200390BE
:108F100000200490059002A91948FDF7E5FE012004
:108F2000C0020290002003900220049002A914487D
:108F3000FDF7DAFE9120000202900120039000204C
:108F40000490059002A905200007FDF7CDFE8020C2
:108F50000290002003900120049002A90848FDF728
:108F6000C3FE002201210520FEF734FA0520FEF79A
:108F700025FA07B000BD0000001002400106000005
:108F80000004005008300000000011100000211003
:108F90000836000010B50A480A49086000204860F9
:108FA0000021084881600849416100210162416255
:108FB0008162FEF725F9002801D0FCF75DFE10BDA7
:108FC000007C00408C160020FFFF000010B5124806
:108FD00012490860FF200530486000210F48816079
:108FE000C160016141610121490281610021C161CA
:108FF0000162416281620721C162FFF705F8002822
:1090000001D0FCF739FE054800680068402108439C
:1090100002490968086010BD00300140BC160020FC
:1090200000B585B014216846FCF7D5F819481A49EF
:109030000860E12040024860002117488160C1605B
:1090400001610C21416100218161C1610162302017
:1090500011494862012109030F4881634900C16336
:10906000FFF754F9002801D0FCF706FE012080022A
:109070000090022001900120029003200390042020
:109080000490694605200007FDF72EFE01F000FE62
:1090900005B000BD003801401417002070470000E3
:1090A00010B5002819DA1A4A03071B0F083B9B0862
:1090B0009B00D2588307DC0EFF23A3409A438B0703
:1090C0001B0E8407E40EA3401A43114B0407240F20
:1090D000083CA408A4001A5118E00E4A03231B02FE
:1090E000D21883089B00D2588307DC0EFF23A340CD
:1090F0009A438B071B0E8407E40EA3401A43054BCB
:10910000032424021B198408A4001A5110BD000076
:109110001CED00E000E100E000BF00BF00BFBFF3B6
:109120004F8F00BF00BF00BF06480749C86000BF9F
:1091300000BF00BFBFF34F8F00BF00BF00BF00BF25
:1091400000BFFDE70400FA0500ED00E0F0B593B0C4
:1091500000200E90962002F069FC4B20C00002F027
:1091600081FC0020FE490870FE4800780C2802DBD4
:109170000B20FC4908700122510205200007FDF771
:10918000B6FEF8480078F8490870F6480078F749C4
:1091900008700020F6490870F6490870F648007813
:1091A000F64908710221F648FDF794FE002801D126
:1091B000012000E00020F349097849000843EF4905
:1091C000C871F14801780068401CEF4A1060C8B2CD
:1091D000EA49C870E54800788872E448007842009F
:1091E000EA49E6480B30FBF7DDFF0620E349487209
:1091F0000846E7490A78427049788170DB49097866
:10920000490008460D300022DC4902F02DFDD74907
:109210000978490008460D30002102F039FD02208E
:1092200002F05EFC0020D549C871DA490870DA49BD
:1092300008700120D94908700020D9490870D94820
:10924000FEF76AF8D84908800020C9490870C74865
:109250000078FCF70CFA0646FCF788FA0022D34B9C
:1092600005910490FCF718F90791069002F006F8B2
:109270000022CF4B09910890FCF75CF80B910A9003
:10928000FCF756FAC0B20D900D984001C649098806
:109290004018C8490880084600880121C90388424F
:1092A00004DBC4480088401AC2490880C248C34948
:1092B0000860C3480078401CC1490870B948FEF7EF
:1092C0002BF8C0490880ADE2B648FEF725F8BD4945
:1092D000088033E0B048007800281BD002F062FB21
:1092E000109012991098884214D9119910988842B8
:1092F00010D202F0E3F90020A8490870384602F0C5
:109300008DFB012002F0ECFBAF4908700020A24960
:1093100008701DE0A348FDF7FFFFAA490880084632
:109320000088A4490988884208DBA6480088A1492A
:109330000988A64A8918884200DA09E000210F202E
:1093400002F0CCFAA2490860A24908400028C1D026
:1093500000BF9F480068401C002801D1FFF7DCFED9
:109360009B48006801218903084000287ED08122A3
:10937000D20100210F2002F030FC0021102002F069
:10938000ADFA4006400E0F90002293480F9902F06C
:10939000F5FA002002F066FB002002F012FB8E4876
:1093A000407A07288FD102228C498B48401DFBF759
:1093B0001DFF002887D102F0C8FC894A03C202F0D1
:1093C000ADFC884A03C26A480078401C68490870AE
:1093D0008148427808A90A74807848746248007805
:1093E000002810D10120804908706846008E674926
:1093F000088001205D490870604908A8007C487019
:1094000008A8407C8870614800886946098E8842B7
:109410007ED176497048C089088075486E49098AAE
:1094200001806048FDF778FF664908807048008831
:10943000FF30C3306E490880084600886D49884275
:1094400012DD6B480088401A694908806748008827
:10945000401C664908800846008866490B318842EE
:1094600002DB002061490880002600E0CEE10320F5
:10947000614988556149584842890A8080894880F5
:1094800008460068B1005E4A50505348C07C00074F
:10949000000F032805D05048C07C0007000F354955
:1094A00008704D48C07C001156490870002044499E
:1094B00008700120384908704049474842890A80AD
:1094C0008089488029480078FF2191314843FF3046
:1094D000FF30FF30F5300004C117424B0CCB801831
:1094E00059410906070A0F434748381A12901920B4
:1094F0008002381811907908490000200A0E0002F5
:1095000010430B02002211469A1848413F4900E0DF
:1095100004E10A60486032480CC818480A3002F07A
:10952000E3FB30480CC81548163002F0DDFB374825
:109530000CC81248123002F0D7FB08200F494872BD
:109540003048007800286FD0022224492248401D6C
:10955000FBF74CFE002867D101200E49087057E048
:10956000E90000202A010020290100202801002014
:109570000901002036010020500100203012002097
:10958000000400502E0100206C0000202A1400204E
:10959000020100202C0100201C0100201E010020DF
:1095A0001D0100208C160020220100200000E03F59
:1095B0000000084024010020A086010004010020D2
:1095C0001901002020010020E8000020983A000046
:1095D0007000002000D027248012002044010020C9
:1095E00078000020800000201B0100204C0100209A
:1095F000F4000020E7030000EC140020F800002035
:109600005C14002037010020005203008800002075
:10961000FD49C8710F981638FC4908700846027851
:10962000FB49FC48FBF7BEFDFB4909788900084669
:109630001C300022F44902F017FBF7490978890031
:1096400008461C30002102F023FB0120F34908707A
:109650000422EF491339F248FBF7A4FDF1480088D2
:109660007D21C9004843F04909884018EF49086046
:10967000EF480078EF490870EF49C888FBF7F7FF1B
:109680000990E8480088FBF7F2FF08900999FBF77A
:1096900013FE7F21C9050A90FBF7B5FD0B90FCF77F
:1096A0000FF8E3490880E3480078401E09888842A3
:1096B00002D10120D9490870DA480088DF490880C2
:1096C000DF490020085EFBF7D9FF09910890DD48CB
:1096D0000088FBF7E7FFDC4ADC4B01910090FBF7C9
:1096E000DBFE05910490D1480068FBF7C7FF0391AA
:1096F0000290059B049AFBF7C1FE07910690099B17
:10970000089AFBF717FE0B910A90FBF7EDFFD04983
:109710000860D048008800F009FD76E06846008EB9
:10972000FCF7E6FB0646CC4909788E4213DB0120A4
:10973000CA490870B8480078401CB74908706846A4
:10974000008E7100C64A5052AF4908A8007C48708C
:1097500008A8407C88700320C2498855C249AC489B
:10976000143842890A808089488008460068B10020
:10977000BE4A5050A6481438C07C0007000FBC49B0
:10978000097888420BDDA2481438C07C0007000F1E
:10979000032804D09E481438C07CB5490870B548E9
:1097A0000078002816D00222B34999480F38FBF7F9
:1097B0001DFD00280ED10120B04908709249C871E2
:1097C0000F981638914908700846027890499148D8
:1097D000FBF7E8FCB00016308B4940180B90A84806
:1097E0000CC80B9802F080FA8B490978890008466A
:1097F0001C300022844902F037FA87490978890031
:1098000008461C30002102F043FA0BE09D4A00217B
:109810000F2002F0E2F99C480078002802D00020D6
:1098200002F0CFF88748008898490988884200DA12
:109830004AE58448008895490988954A89188842EC
:10984000F6DC904A00210F2002F0C7F99148007819
:1098500071490870002583480078002818D17048A5
:109860000068FCF72DFC8C49088008880988491E8F
:10987000894B198089490988FBF750FC8848008882
:10988000414388B2734908800846008800F04EFCC6
:10989000002084490870002423E07248005D0028FD
:1098A0001DDD80480078401C7E4908706D48005DD1
:1098B000A9007D4A505060006949085A69007B4AF6
:1098C0005052A00069490A582946681CC5B2880050
:1098D00077490A506348005D401E62490855601C84
:1098E000C4B25D4800785D4909784018A042D4DCD4
:1098F00068480078032803DA6A48007869490870E4
:10990000684800785449087000243FE0002536E09C
:10991000A80067490958681C8000654A10588142B0
:109920002BDDAA00624B99586A00604B985AA2003E
:109930005D4B9A580C926A1C92005D4B9A58AB0092
:109940005B4EF2506A1C5200584B9A5A6B00574EAD
:10995000F2526A1C9200544B9A58AB00524EF2508D
:109960006A1C9200524B99506A1C52004F4B9852FD
:109970006B1C9B000C9AF25000BF681CC5B23648A5
:109980000078401EA842C3DC601CC4B23248007894
:10999000401EA042BADC002046490870002496E030
:1099A00060004249085A61002D4A5052A0004049C7
:1099B0000858A1002D4A5050A000114608583E49B1
:1099C00088427DD0A000384908580A287DD13948FE
:1099D000007806214843001D384940186100204A9C
:1099E00089180A78027049784170A2001F4BD1187B
:1099F000304A127806235A43921D304BD018042265
:109A0000FBF7D0FB2B485CE0301200202D0100203A
:109A100094120020F8140020280100201D010020CD
:109A2000300100204C010020F40000200C01002037
:109A30006C0100202B010020BC0D0020260100201D
:109A40003401002020010020F853E3A59B843E4010
:109A50001401002052010020290100201B010020D8
:109A60002A140020EC140020F80000205C140020D0
:109A70003601002037010020440100202C01002085
:109A80008000002000D027241E0100202401002097
:109A9000983A000009010020FC0000205801002035
:109AA000560100202A010020BC140020421400208E
:109AB0008C1400201A010020FFFF0100DE1300209B
:109AC00003E00078401C21490870601CC4B22048A3
:109AD0000078844200DA63E7002405E01D48A10015
:109AE0001D4A5050601CC4B20C2CF7DB1B48007898
:109AF00000281CD000200C9000260B9018480078FD
:109B00000B901748467880780C900B9802280DD15E
:109B1000144988191249C91C0C9AFBF743FB02F03F
:109B20006BFA642001F00EFCFFF7F6FA00BF0E4A54
:109B300000210F2002F051F80022012149020520E6
:109B40000007FDF7D4F913B0F0BD00001A010020A2
:109B500029010020FFFF01005C1400202C010020DF
:109B6000F8140020BC0D002080D02724704700008E
:109B7000FEB5AC4802900020C0430190002796201B
:109B800001F054FF4B20C00001F06CFF0020A649FB
:109B90000870002622E1A5488673002201461420A1
:109BA00002F062F80021142002F072F8022001F0A5
:109BB00097FF00BF00210F2001F090FE9C49086034
:109BC0009C4908400028F5D099480068401C0028AE
:109BD00001D1FFF7A1FA96480068012189030840E6
:109BE00000287DD08122D20100210F2001F0F5FF55
:109BF0000021102001F072FE45066D0E294600225C
:109C00008D4801F0BBFE8C48407A022869D10222BF
:109C10008A498948401DFBF7E9FA0028F6D102F08D
:109C200094F8874A03C202F079F8864A03C2002FEB
:109C30002BD1012784498048C089088083487E4908
:109C4000098A01808248FDF767FB824908807F48C6
:109C50000088FF30C3307D490880084600887E496F
:109C6000884212DD79480088401A78490880764891
:109C70000088401C744908800846008876490B31EA
:109C8000884202DB0020704908806B48428969469F
:109C90000A808089488004226749491C6F48FBF785
:109CA00081FA684803684068FF22520400219A182C
:109CB00048410106140A0C43204601F0AFFE61083A
:109CC000490000200A0E000210430B020022114638
:109CD0009A18484162490A60486059480CC801E036
:109CE00072E06DE05D48093001F0FEFF55480CC898
:109CF0005A480D3001F0F8FF59480CC85748113048
:109D000001F0F2FF00225549491E3C2001F0ACFF52
:109D100000213C2001F0BCFF012001F0E1FE51498F
:109D2000087041480078401C3F4908700121C90370
:109D300005200007FCF7F2F84B480068FCF7C0F973
:109D40004A49088008880988491E484B19804849B3
:109D50000988FBF7E3F947480088414388B2464940
:109D600008800846008800F0E1F9009902988142D5
:109D700010DA009800280DD004222F49491C01A8B0
:109D8000FBF710FA01203D49087005203C49087096
:109D90000098029033480078002808D100BF0021C5
:109DA0000F2001F09BFD802108400028F7D0802281
:109DB00000210F2001F011FF0020324908700BE054
:109DC00001203049087007E02F4A00210F2001F0E0
:109DD00004FF01202B490870701CC6B2032E00DA64
:109DE000D9E6002F1AD121480088401E1F4908805B
:109DF00008460088002805D0084600881C490988C4
:109E0000884203DD1A4800881849088017480088EE
:109E1000401E184909884843174908801B49019882
:109E20000880FEBD3F420F00E9000020BC11002069
:109E30007000002000D02724801200204401002060
:109E400078000020800000204C010020F400002059
:109E50008C16002020010020E7030000DF11002005
:109E600088000020E800002030010020FC000020D5
:109E700058010020560100205201002060000020FF
:109E800008010020BC0000200090272402010020CF
:109E9000F8B549484949086002F03AF80120400203
:109EA000474948800020C8876420C8800846C08889
:109EB000002801D16420C88042480078432802DD90
:109EC0004320404908703F480078002802DA00200B
:109ED0003C4908703A48C08E3A4908703848C08FEB
:109EE000394908703648808F384908703448807A7C
:109EF000374908703248808836490860052036495D
:109F000008802F49C88834490988FBF707F9334985
:109F100008802B49888831490988FBF7FFF82E48CB
:109F20000088414388B22E49088009887D22D200EA
:109F300051430846FBF7A2FB04462A4A2A4BFBF78B
:109F400013FB0646FBF7F4FB2849088024480088E9
:109F5000274908801A48C1887D20C000FBF7DEF839
:109F6000244908801648C1887D20C000FBF7D6F838
:109F700021490880012021490880FBF7D7FF2049AB
:109F800008801A4802881F491F48FDF7C9F90028B0
:109F900001D0FBF771FE0F4801681CA000F08AFF9A
:109FA0000748C1881DA000F085FF0548018920A051
:109FB00000F080FFF8BD0000D9AC00084800002088
:109FC000BC0D002001000020660100206701002078
:109FD0004F010020440100205601002058010020BC
:109FE00052010020F853E3A59B843E405E0100200F
:109FF00062010020600100206A0100206C01002045
:10A0000064010020FF7F00008C160020B1EAC7A980
:10A0100049443A202564202E0D0A0000CDA8D1B66F
:10A02000BCE4B8F43A202564206D732E0D0A0000BC
:10A03000B5A5B4CECDA8D1B6BBF9D5BECAFDC1BFBA
:10A040003A202564B8F62E0D0A00000000B585B050
:10A0500014216846FBF7BFF800220121C90310480C
:10A06000FCF745FF0120C003009001200190002073
:10A070000290039069460A48FCF736FE0120C003AF
:10A08000009003200190002002900390694604484C
:10A09000FCF72AFE022001F055F905B000BD0000D2
:10A0A000000400507047000038B504460D460020FB
:10A0B000009055201B490870AA2048700320887022
:10A0C000601DC870032008710846457184716800DE
:10A0D000154A811822461348C01DFBF763F800207B
:10A0E00008E0811C0F4A525C6946098851188AB2FF
:10A0F0000092401C611D8842F3DB0A48801CFBF77C
:10A1000007FD0090E01D0749411868460078087077
:10A1100068464078487021460931024800F03AFB11
:10A1200038BD0000CC150020BC0D0020F0B585B076
:10A1300005461A4800881A490988884206DB1748EC
:10A14000008817490988401A144908801548C088B2
:10A1500012490988484347197D21C9004F431248D5
:10A1600000683E1A3046FBF789FA104A104B0191FD
:10A170000090FBF7F9F903910290FBF7B5FA04465A
:10A180000C498C4201DD0846241A002C01DA0948EA
:10A19000241809480068446105B0F0BD6C01002036
:10A1A0006A010020BC0D002014010020F853E3A533
:10A1B0009B843E40FF7F00008C160020014600205B
:10A1C000054A126890B2054A104002460A431046FA
:10A1D000014A10607047000000300140C7FF0000D6
:10A1E00010B5FCF791FE10BD00B599B034210CA854
:10A1F000FAF7F1FF142107A8FAF7EDFF1C216846D2
:10A20000FAF7E9FF244800680321C90288430121C5
:10A21000C902401820490860FDF7EEF81F480069A0
:10A220000321C90288431D49086106200C90881546
:10A230000E9001200F901020109002201590002108
:10A24000169141041791410518910CA8FDF7CAFB1E
:10A25000002801D0FBF710FD0F2007900320089085
:10A26000002009900A900B90012107A8FDF724FA1D
:10A27000002801D0FBF700FD812000900020029013
:10A280000320800406906846FDF700F9002801D0FD
:10A29000FBF7F2FC19B000BD007000404010024016
:10A2A00015480068FF21013108431349086008463A
:10A2B000C068124908401049C86008460068104943
:10A2C00008400D49086008468068400840008860E2
:10A2D0000846006801218904884307490860084648
:10A2E000C068FD21090488430349C8600020086153
:10A2F0000448054988607047001002400C40FF8800
:10A30000F6FFF6FE0050000800ED00E010B501F089
:10A31000FFFA044602E001F0FBFA04460D488442CD
:10A32000F9D100200C4908800C480078002804D09E
:10A33000012805D0022809D105E0FFF719FC05E046
:10A34000FBF716FE02E0FEF701FF00BF00BF01F0C1
:10A3500099F910BD3001CADEE6000020600000203F
:10A36000818CC907C90F002908D0016849680122FA
:10A3700052049143826A1143026851600222416A89
:10A380001140022907D101684968D2039143C26A8A
:10A390001143026851600422416A1140042907D127
:10A3A0000168496812049143026B114302685160CD
:10A3B0000822416A1140082907D10168496812033F
:10A3C0009143426B1143026851601022416A11406F
:10A3D000102907D10168896812029143826B1143E9
:10A3E000026891602022416A1140202907D101684A
:10A3F000896812029143C26B114302689160402246
:10A40000416A1140402915D101684968920391437E
:10A41000026C11430268516001221205016C9142E5
:10A4200008D101684968032252059143426C1143E7
:10A43000026851608022416A1140802907D1016879
:10A44000496812039143826C11430268516070475E
:10A4500038B504460020E067FCF750FD054620684B
:10A4600000680821084008280BD114482B46002218
:10A4700089040090204600F0C9FB002801D0032089
:10A4800038BD206800680421084004280BD10B481F
:10A490002B46002209050090204600F0B7FB00285B
:10A4A00001D00320ECE720206067A06700BF0021F7
:10A4B0007020015500BF0020E2E70000FFFFFF0110
:10A4C00070B50025C82420480078002800D070BD51
:10A4D0001E480078002800D0F9E701201B490870C9
:10A4E0001B48406B002801D10870F0E71848406B0A
:10A4F000C8210D1A1CE01749174A1268885C1749D1
:10A5000009688847164800880A2148431549088089
:10A5100011480068401C1049086008460068C828B7
:10A5200001DB002008600A48406BC8210D1A641E38
:10A5300009480068A84201D0002CDCDC0020034957
:10A54000087000BFC3E70000420000204400002064
:10A5500000000240F40C00203800002048000020D9
:10A56000600100207401002010B53A4800780028EE
:10A5700003D139480078002800D010BD01203649A9
:10A5800008703648C06980210840002802D132494D
:10A590000870F2E7324900200856324900228A56F4
:10A5A000904215D12D48C0694021084000280BD0A9
:10A5B0002D480078002807D000202B4908702B4830
:10A5C0000088401C29490880002023490870D4E7EE
:10A5D00025480078002805D10120234908700A2069
:10A5E00000F0BAFE1F4900200856CC2148432049FC
:10A5F0004018001D1F490968405C184988621D48C1
:10A600000068401C1B490860164900200856CC21F0
:10A6100048431749085817490968884214DC002044
:10A62000144908600F480078401C40B20D4908707A
:10A63000084600780E2801D1002008700E480078E6
:10A64000401C40B20C49087000200349087000BF4C
:10A6500093E7000042000020430000200038014042
:10A66000350000203400002045000020520000206A
:10A67000CC010020580000203600002070B50546AF
:10A68000AC6A00215A200153522001532046FDF7A5
:10A6900056FD70BDF8B50546AC6A666FA76F2068B9
:10A6A000806880210840802807D1212E05D1002113
:10A6B00052200153204600F064F820688068402151
:10A6C0000840402807D1222F05D100215A200153EC
:10A6D000204600F034F8E06F10210843E067204680
:10A6E000FDF72DFDF8BD70B50546AC6A2868006819
:10A6F00020210840002817D100215A20015320684A
:10A700000068FF2101318843216808602068806863
:10A7100040084000216888602068806840218843A4
:10A72000216888602020A0672046FDF721FF70BDCA
:10A7300070B50446A56A2846FDF71BFF70BD016889
:10A740000968FF222132914302681160016889681B
:10A750004908490002689160202181670021016653
:10A76000704710B50446206800684021884321687E
:10A77000086020206067002060662046FDF77AFFB1
:10A7800010BD01680968C022914302681160202150
:10A790004167704770B505460C4620480078002890
:10A7A00003D11F480078002800D070BD01201B494C
:10A7B0000870C82C04DC1B4800214156002903DC2A
:10A7C000002016490870F0E7174900200856CC21F0
:10A7D000484316490C50144A00215156CC2251438B
:10A7E000124A8918081D22462946FAF7DBFC0E4852
:10A7F0000078401C40B20C490870084600780E28CA
:10A8000001D10020087007480078401E40B2054979
:10A81000087000200149087000BFC6E74200002010
:10A82000430000203600002035000020CC0100202D
:10A83000F0B587B004461020049000250020039056
:10A840000026E7492068884200D100E000BF216966
:10A85000A068084361690843E16908430746206826
:10A860000068E04908403843216808602068406873
:10A87000032109038843E168084321684860A76908
:10A88000D7492068884201D0206A07432068806841
:10A890000B210902884338432168886000BFD249F0
:10A8A000206888421CD1D148C0688007800F0028EA
:10A8B00006D001280AD0022805D003280CD108E0D0
:10A8C000012004900BE00220049008E00420049092
:10A8D00005E00820049002E01020049000BF46E04C
:10A8E000C349206888421CD1C048C0680C21084078
:10A8F000002806D004280AD0082805D00C280CD13E
:10A9000008E0002004900BE00220049008E00420FE
:10A91000049005E00820049002E01020049000BF9D
:10A9200025E0AF49206888421FD1B048C0680321A4
:10A9300089020840002808D001218902401A0AD063
:10A94000401A05D0401A0CD108E0002004900BE01A
:10A950000220049008E00420049005E00820049000
:10A9600002E01020049000BF01E01020049000BF1E
:10A970009B492068884256D1049804281AD004DCE8
:10A98000002807D002281CD108E0082816D010287B
:10A9900017D117E0FCF79AFF064616E093484038B7
:10A9A0000068102108400009002801D0914E00E005
:10A9B000914E0AE0FCF7AEFF064606E00126F603DC
:10A9C00003E000BF0120039000BF00BF002E0AD0AB
:10A9D000606841004018B04203D860680003B0428C
:10A9E00002D201200390F4E0606802903046FF211B
:10A9F000013100F086FA626852080023801859413C
:10AA000001910090029AFAF79DFB0546032000028F
:10AA1000854205D37948854202D82068C560D8E0D0
:10AA200001200390D5E00121C903E06988426FD17C
:10AA3000049804283CD006DC002809D0012813D053
:10AA400002284AD11CE008283ED0102845D145E014
:10AA5000FCF73CFF400061684908401802906168BB
:10AA6000FAF746FB85B23CE0FCF742FF4000616824
:10AA70004908401802906168FAF73AFB85B230E065
:10AA80005A4840380068102108400009002807D0C3
:10AA900061684A085A4BD018FAF72AFB85B206E0DB
:10AAA00061684A08574BD018FAF722FB85B218E0C4
:10AAB000FCF730FF40006168490840180290616867
:10AAC000FAF716FB85B20CE061684A0801231B0403
:10AAD000D018FAF70DFB85B203E000BF0120039008
:10AAE00000BF00BF102D0FD3474885420CD8464801
:10AAF0000F38284005902807400F05990843059016
:10AB000005982168C86064E00120039061E0FFE7D8
:10AB1000049804283AD006DC002809D0012812D075
:10AB2000022847D11AE008283BD0102842D142E041
:10AB3000FCF7CCFE61684908401802906168FAF79A
:10AB4000D7FA85B23AE0FCF7D3FE616849084018AD
:10AB500002906168FAF7CCFA85B22FE023484038BA
:10AB60000068102108400009002807D061684A08E1
:10AB7000204BD018FAF7BCFA85B206E061684A08A3
:10AB80001D4BD018FAF7B4FA85B217E0FCF7C2FEF5
:10AB900061684908401802906168FAF7A9FA85B21D
:10ABA0000CE061684A080123DB03D018FAF7A0FA29
:10ABB00085B203E000BF0120039000BF00BF102D4D
:10ABC00005D31148854202D82068C56001E0012004
:10ABD0000390002020666066039807B0F0BD000077
:10ABE00000480040F369FFEF003801404010024088
:10ABF0000044004000093D000024F400FFFF0F0066
:10AC000000127A000048E801FFFF0000FFB581B0A4
:10AC100004460D4617460A9E22E0701C00281FD0ED
:10AC2000FCF76CF90499401AB04201D8002E17D1F4
:10AC300020680068FF21A1318843216808602068EE
:10AC40008068400840002168886020206067A06715
:10AC500000BF00217020015500BF032005B0F0BDEA
:10AC60002068C0692840A84201D1012000E00020EE
:10AC7000B842D2D00020F1E710B51020034909688E
:10AC800008620248FDF75CFA10BD000014170020AE
:10AC90000D200149087070473600002010B50A48A1
:10ACA00000880A21484309490880FEF779F8FEF731
:10ACB000B7F9C82206490748FDF7E6FB002801D08E
:10ACC000FAF7DAFF10BD00006001002074010020D7
:10ACD000F40C00201417002070B5044600256A48C3
:10ACE0000078082865D100BF002004E06749095CAE
:10ACF00049198DB2401C66490978491F8142F5DC2B
:10AD000064480078281885B261480078281885B210
:10AD100061480078281885B260480078281885B204
:10AD20005F480078281885B26019C007C00F002856
:10AD300035D058480078012827D002282DD159490C
:10AD4000554A1278881855490A785049FAF72AFA6C
:10AD500001F052F9642000F0F5FA00BF00BF00BF17
:10AD600000BF00BFBFF34F8F00BF00BF00BF4E4802
:10AD70004E49C86000BF00BF00BFBFF34F8F00BF88
:10AD800000BF00BF00BF00BFFDE74348007841108F
:10AD900042480078FFF788F900E000BF00BF0020BC
:10ADA000394908703C4908703949087040490870B1
:10ADB00068E035480078072812D134483C490978C2
:10ADC00044543B480078401C3949087030480078AA
:10ADD000401F0978884255D108202B49087051E05E
:10ADE00029480078062805D12C48047007202649F8
:10ADF000087047E024480078052805D126480470EB
:10AE00000620214908703DE01F480078042805D13C
:10AE10002048047005201C49087033E01A48007867
:10AE2000032808D11A48047000201B490870042028
:10AE30001549087026E014480078002805D1552CE3
:10AE400003D10120104908701CE00F480078012848
:10AE500005D1AA2C03D102200B49087012E00A4840
:10AE60000078022807D1032C05D103200649087079
:10AE70000B48047006E0002003490870064908707A
:10AE80000349087070BD00003A01002068150020D9
:10AE90003C0100203F0100203D0100203B0100203B
:10AEA0003E010020BC0D00200400FA0500ED00E08A
:10AEB000400100200FB410B503A9044B044A0298C6
:10AEC00000F034F910BC08BC04B0184705BD0008F8
:10AED0008C0100202021020C01D010211046020A12
:10AEE00001D010460839020901D01046091F820816
:10AEF00001D01046891E420801D0881E7047081AEA
:10AF00007047F8B582B28BB2040C0D0C1046584352
:10AF1000002126465E43370C3604801979411646D7
:10AF20006E43370C36048019794126466E438919E1
:10AF3000F8BD30B47446641E2578641CAB4204D35B
:10AF4000635D5B00E31830BC18471D46F8E702E07C
:10AF500008C8121F08C1002AFAD1704770470020A4
:10AF600001E001C1121F002AFBD1704708B5002182
:10AF700000916B46012202212C2000F043FE0221A9
:10AF800000916B4601222C2000F03CFE08BD000021
:10AF900038B504466D2000906B46012208492E20EA
:10AFA00000F030FE002C05D0064A07492E2000F0A4
:10AFB00003FE04E0054A04492E2000F0FDFD38BDE3
:10AFC000060800000706000006180000071600002B
:10AFD00038B504466B4602220021362000F09EFC64
:10AFE0002300FFF7A6FF0E11081A545454542331BE
:10AFF00054543D444B540021684601704078FE2172
:10B0000008406946487043E069460878FC210840DA
:10B0100001210843694608703AE069460878FC2136
:10B020000840022108436946087031E0684600780C
:10B03000B3210840482101436846017040788021CF
:10B0400008436946487023E068460178B320014010
:10B050006846017040784106490E6846417017E025
:10B0600069464878022108436946487010E06946FD
:10B070004878FD2108406946487009E0694608782B
:10B08000CF210840202108436946087000E000BF36
:10B0900000BF6B4601220021362000F0B3FD00AB5B
:10B0A000013301221146362000F0ACFD38BD08B551
:10B0B000032168464170012101706B460222002184
:10B0C000362000F09FFD0122D20306212D2000F042
:10B0D00073FD012000F036F90120FFF779FF08BD6C
:10B0E00038B504462004010E6846417004706B4672
:10B0F000022204212D2000F085FD03216846017005
:10B100006B46012206212D2000F07CFD00216846BF
:10B1100001706B46012206212D2000F073FD0A21EB
:10B120002D2000F0DBFB0546284638BDFFB58DB06D
:10B130000446002506E025280AD0109A0F9990476A
:10B14000641C6D1C20780028F5D1284611B0F0BD94
:10B1500000270121484A009700E00743641C237838
:10B160000846203B98401042F7D120782E2817D16E
:10B17000042007436078641C2A280CD10E98641CB4
:10B1800002C800910E900BE000990A225143303919
:10B190004018641C00902078014630390929F3D901
:10B1A00020780028D1D0642808D0692806D07528D6
:10B1B0001ED0109A0F9990476D1C5BE00A200E99E3
:10B1C000019001C90E91002802DA40422D2102E0CF
:10B1D000390504D52B216A461172012103E0F907D4
:10B1E00004D02021F7E70BAE0B910DE00021FAE728
:10B1F0000A200E99019001C90E91F7E70199F9F71C
:10B2000077FF3031761E31700028F7D103A8801BFC
:10B2100020300190780701D5009801E001200090CE
:10B220000199884201DD401A00E0002000270090CB
:10B2300006E002A8109AC05D0F9990476D1C7F1C14
:10B240000B988742F5DB04E0109A30200F99904765
:10B250006D1C0099481E00900029F5DC05E030784F
:10B26000109A761C0F9990476D1C0199481E019009
:10B270000029F4DC641C65E709280100F8B54A00E0
:10B280002B4B520DD6182B4A0C460546142E2BDAA2
:10B29000002E12DA284BFAF74DF800221346FAF77F
:10B2A00079FA40D2002C03DA0124E40700253AE0C1
:10B2B0002046284337D0214C14E0214F0B46F7405D
:10B2C0003B402B4331D01C4BFAF734F80022134695
:10B2D000FAF760FA27D2002C03DD01200005F040C8
:10B2E0000419BC4300251EE0332E1EDC3346002724
:10B2F000143BFF43DF40384217D00F4BFAF7C4F836
:10B3000000221346FAF746FA0DD2002C0ADD142E5D
:10B310000CD03420811B012088404019A84200D263
:10B32000641C0546BD4321462846F8BD641CF9E768
:10B3300001FCFFFF9C7500883CE4377E0000F03F75
:10B34000FFFF0F0070B504467D20C0006043054636
:10B35000284600F001F870BD002100BF40E000BFAA
:10B3600000BF00BF00BF00BF00BF00BF00BF00BFE5
:10B3700000BF00BF00BF00BF00BF00BF00BF00BFD5
:10B3800000BF00BF00BF00BF00BF00BF00BF00BFC5
:10B3900000BF00BF00BF00BF00BF00BF00BF00BFB5
:10B3A00000BF00BF00BF00BF00BF00BF00BF00BFA5
:10B3B00000BF00BF00BF00BF00BF00BF00BF00BF95
:10B3C00000BF00BF00BF00BF00BF00BF00BF00BF85
:10B3D00000BF00BF00BF00BF00BF00BF00BF491CCF
:10B3E0008142BCD370470000F0B585B00446002010
:10B3F000049003902578607940008A49085A0290A9
:10B400006078401E8849C6B20863042D01D0072D1C
:10B4100001D1012000E000200190207882490873CA
:10B42000E07900280AD1084680690121890508438E
:10B430007D4988610298C010029006E07A488069D0
:10B4400001218905884378498861207A76494873C3
:10B4500008468069217A0904032212041140084336
:10B4600071498861084600218269042000F0B5FB1B
:10B470006E492E20029A00F09FFB3046FFF788FDB0
:10B480006B48405D810040186A4943180522072136
:10B490002B2000F0B7FB684901980B1801220B2103
:10B4A000282000F0AFFB6248405D800063490A58E5
:10B4B0000C21282000F091FBE079800060494018C1
:10B4C000A1794900425A0221272000F075FB700043
:10B4D0005C490A5A0421272000F06EFBE07900281D
:10B4E00005D164220621272000F066FB1EE0A0782B
:10B4F00004280DD11020009010220621272000F0F2
:10B500005BFB6B4601222621272000F07BFB0DE030
:10B510002820009020220621272000F04DFB6B46BA
:10B5200001222621272000F06DFB00BF3001464993
:10B530004018E178890042580821272000F04DFB8F
:10B54000A17A627A08021043002803D13F49617250
:10B55000090AA172A17A637A0802184302462021DF
:10B56000272000F029FB3A480C210268232000F034
:10B5700034FB71003648001D425A0421232000F09C
:10B580001BFBA07900280BD0E07932494318012237
:10B590000021212000F036FB0320049001200390BD
:10B5A0002807000F2901F02211400843617889041F
:10B5B00003229204114008430499090592001140A6
:10B5C0000843039949040122520411400843217998
:10B5D00089051F229205114008436179C906C90EE9
:10B5E000C906084307463A4600211F2000F0F5FA35
:10B5F000A0786178084300040B4908610846006997
:10B60000E17949030122D203114308430649086145
:10B61000084600210269082000F0DFFA002005B08A
:10B62000F0BD0000E8C000089001002004280000E0
:10B6300090C00008020000202000002098C00008F0
:10B64000B8C00008C4C00008C8C00008411000000D
:10B65000B0C000082200002038B504460D46084856
:10B66000808B0443224600212C2000F0A5FA00958F
:10B670006B46012206212C2000F0C4FA38BD0000E0
:10B680009001002010B5FFF771FC10BD70B50546A4
:10B690000421362000F022F90446002D03D00120B9
:10B6A000C002044304E00121C90220468843044645
:10B6B00022460421362000F090FA70BD38B54020B3
:10B6C000009000210E2000F009F9044600221146E6
:10B6D0000E2000F082FA6B46012200210D2000F0BE
:10B6E00091FA084A00210F2000F077FA00F048FA9A
:10B6F000224600210E2000F070FA0021024801735A
:10B7000038BD0000F8FF2724B0010020F0B585B057
:10B710000646042002900027002001905F494875EA
:10B72000086300215D4820304171017300205B49AE
:10B7300088834863886300F0EBF85849086003E0A9
:10B7400000F0E6F8554908605448006854498842BA
:10B75000F6D10020FFF73CFC52480078242804DD95
:10B76000504800780446243C0DE006214D480078FE
:10B77000F9F7D4FC0621081A45014A480078F9F780
:10B78000CDFC2C460C43200621040843210208432B
:10B790002043039000211E20039A00F01EFA02AB02
:10B7A00001220021242000F02DFA1E20FFF798FC32
:10B7B00087B23812394988730420FFF791FC019051
:10B7C0000198C0B200280FD0022000906B460122E1
:10B7D00012212D2000F016FA3048808B0121090338
:10B7E00008432E49888300BF00F092F82B49086077
:10B7F0000620FFF775FC294948600720FFF770FC19
:10B8000026498860F806C00E08750846007D0028A5
:10B8100001D1102008752149087D00F04BFAF0078E
:10B82000C00F002809D0FFF742FC1C48808B012183
:10B83000C9020843194988830CE00521362000F02D
:10B8400035F80546184805402A460521362000F0FF
:10B85000B3F900BF0120FFF7BBFB0021042000F07B
:10B860003DF80E4988610021262000F037F8054692
:10B87000052080030543800005432A460021262039
:10B8800000F0ABF900222621362000F095F900F0F7
:10B890003FF802490860002005B0F0BD900100208B
:10B8A0003001CADE01000020FFFD0000F8B50446AB
:10B8B0000D46094FA9B2A0B26B46022200F02EF845
:10B8C0000646002E06D16846407801026846007898
:10B8D000081887B23846F8BDFFFF0000FEB50546E0
:10B8E0000E460027FF43B1B2A8B201AB042200F01C
:10B8F00015F800900098002808D1032404E03802CD
:10B9000001A9095D4718641E002CF8DA3846FEBD0F
:10B9100010B500210846FFF7E1FF10BDFFB581B06B
:10B9200006460C4617460025002C04D129466D1CFE
:10B93000684646541AE040203043C2B229466D1C86
:10B94000684642547F2C04DC28466D1C69460C5422
:10B950000CE0E0B28021084329466D1C6A46505431
:10B960006004020E28466D1C69460A54A8B23A4685
:10B970006946049B00F00CFB05B0F0BD70B50446B1
:10B980000D46164623462A4631461120FFF7C6FFCC
:10B9900070BD10B504462346052200211520FFF78F
:10B9A000BDFF10BD10B501210620FFF797FF10BDA8
:10B9B00010B504462346052200211720FFF7AEFFED
:10B9C00010BD38B504460020009000F0D9F8FF25DE
:10B9D0000135002C01D0680005432A4600210D20C6
:10B9E00000F0EAF8002C17D06B46012203210F204B
:10B9F000FFF794FF684600780821084000280BD024
:10BA0000FFF75CFEFF2501352A4600210D2000F0DE
:10BA1000D3F80020C04338BD0020FCE710B5044631
:10BA2000224601210A2000F0D8F810BD70B5054665
:10BA300000211A20FFF752FF0446240D2405280395
:10BA4000000B0443224600211A2000F0C6F870BD06
:10BA500010B50446224602492E2000F0ADF810BD74
:10BA60000418000038B504466B4601220321042067
:10BA7000FFF754FF002C16DD224600210C2000F0B9
:10BA80009BF8694608781021084300900F488069A8
:10BA9000090608430D4988616B46012203210420F1
:10BAA00000F0B0F810E06946087810218843009053
:10BAB0000648806909068843044988616B4601226B
:10BAC0000321042000F09EF838BD00009001002002
:10BAD00010B5044622460021182000F06DF810BD74
:10BAE000F8B50446002500200090002602202040E2
:10BAF00000280AD0802000906B46012200210D20F2
:10BB000000F080F801211D480173E007C00F0028F4
:10BB100026D0694608780621084300906B4601222A
:10BB200000210D2000F06EF803210F20FFF7BEFE6C
:10BB300006468120C0003040002801D100251AE0CF
:10BB4000402000906B46012200210D2000F05AF8A1
:10BB50000020FFF79BFD0021084801734D1E0AE0FD
:10BB6000694608780221084300906B4601220021B3
:10BB70000D2000F047F82846F8BD0000B001002075
:10BB80001CB501AB012203210F20FFF7C7FE694658
:10BB9000087980210840694609794022114049000E
:10BBA000884208D0012000906B46012203210D201D
:10BBB00000F028F800BF1CBDF8B505460E46144637
:10BBC0006846047021124170B1B2A8B26B460222DD
:10BBD00000F018F807463846F8BDFEB506460F4691
:10BBE0001446002503E069464C55240A6D1C042DBB
:10BBF000F9DBB9B2B0B26B46042200F003F8019051
:10BC00000198FEBDFFB581B006460C4617460025DB
:10BC1000002C07D180203043C2B229466D1C6846F3
:10BC2000425419E0C0203043C2B228466D1C694618
:10BC30000A547F2C03DC28466D1C0C540CE0E0B247
:10BC40008021084329466D1C6A4650546004020E48
:10BC500028466D1C69460A54A8B23A466946049BB8
:10BC600000F0E4F905B0F0BD70B504460E46154687
:10BC7000281901218902884202DD0020C04370BDDD
:10BC8000A21E334629460920FFF7BCFF0020F6E735
:10BC900070B504460D46064800692043A9050843CF
:10BCA0000646324600210820FFF797FF002070BDAE
:10BCB0009001002038B504466B4601220E212B204E
:10BCC000FFF72CFE68460078410949010091E10622
:10BCD000C90E68460078014300916B4601220E218F
:10BCE0002B20FFF78FFF38BD70B50146002006E01E
:10BCF0000A541E06140A34431B0A2246401C042818
:10BD0000F6DB70BD13B50C4601231A46694602489E
:10BD1000FCF730FC00981CBD141700207CB50021F6
:10BD20000C460D466846FFF734FE042608E0220E56
:10BD300028021043240205466846805D0443761EAF
:10BD4000002EF4DA204629467CBD7CB500210C4645
:10BD50000D466846FFF72CFE042608E0220E280256
:10BD60001043240205466846805D0443761E002E7B
:10BD7000F4DA204629467CBDFBF7CEF8FEF734FA0C
:10BD8000FDF728F8FDF706F9FDF70AF8FDF748F981
:10BD9000FDF71CF9FCF7BCFF0122D10305200007C9
:10BDA000FBF7A5F8FEF774F8FCF77AFEF9F720FF29
:10BDB000F9F7E2FE0721FF204130FFF74DFC2E4846
:10BDC00000880A2148432D490880012211030520DB
:10BDD0000007FBF78CF8C82229492A48FCF754FBD6
:10BDE000002801D0F9F748FF45E0274800780028EF
:10BDF0003FD0FEF7F9F9002023490870FAF7B0F9AF
:10BE000022490870084600780F280DDD0122110331
:10BE10001F48FBF76CF8FEF779FA002201210903AD
:10BE20001B48FBF764F80CE0012251031848FBF7AC
:10BE30005EF8FEF76BFA0022012149031448FBF774
:10BE400056F8FCF72BFD0D480088002804DD0B4850
:10BE50000088401E094908800E48007800280AD151
:10BE600006480088002806D101210846FBF7EAFAB7
:10BE700001E0FCF713FDB8E7600100207401002029
:10BE8000F40C002014170020510100205001002064
:10BE9000000400504500002000B585B01748FBF7AE
:10BEA0000AF914216846F9F796F91548009003201D
:10BEB000019000200290694605200007FAF714FF60
:10BEC00069461048FAF710FF69460F48FAF70CFF69
:10BED00001210846FBF7B6FAFF200130FBF784FA90
:10BEE0000A48006804210843084908608815FBF7E0
:10BEF0008DFAFBF793FA05B000BD00008C16002008
:10BF0000FFFF0000000400500008005000700040D7
:10BF100010B5012292021B491B48F9F7E4FE1948AB
:10BF200000881A4988422CD0084616490880042007
:10BF30008880FF20F530C8800A20088100204881D1
:10BF40001E20C04388810120C88100200884088207
:10BF500048828882C882088388834320C88602205A
:10BF600008877820488701208887C88700210548EE
:10BF7000403001844184818400200249C88300F05C
:10BF80003BF810BDBC0D002000FC0008AA550000C5
:10BF900070B504460D460021102005263607B06214
:10BFA00000BF0DE0685C134EF06000BF1148806870
:10BFB000C007C00F0028F9D00E48C0681870491C8F
:10BFC000A142EFDB00210DE000200A4EF06000BF2F
:10BFD00008488068C007C00F0028F9D00548C0682D
:10BFE0005854491C9142EFD3102005263607B06102
:10BFF000002070BD0030014010B5002472B6012150
:10C0000089020848F9F754FE0446002C06D00122A4
:10C01000920205490348F9F73DFF044662B62046FF
:10C0200010BD000000FC0008BC0D002070B50446E7
:10C030000D460021102005263607B06200BF0CE037
:10C04000685C124EF06000BF10488068C007C00FE7
:10C050000028F9D00D48C068491CA142F0DB00213E
:10C060000CE0585C094EF06000BF08488068C007CB
:10C07000C00F0028F9D00548C068491C9142F0D390
:10C08000102005263607B061002070BD0030014049
:10C090000000010203040005405C0000A05C0400F5
:10C0A000C06C0800805C0400E03F1E00E07D1E00C4
:10C0B00007A9022570889B880A0016000100060067
:10C0C0000100020087008D002D001A3152001A3342
:10C0D0009A001A351D011A376B003B31BE003B3305
:10C0E0005E013B3596023B37000099599959EB5157
:10C0F0008F421E45142E0080EB51F5283333E13A70
:10C10000703DE13AC235852BC2353333C235C23575
:10C11000AE47E13A5138A33051380000000000002A
:10C1200000000102030406070809000000000102E4
:10C130000304030406080C10182030005CC100083A
:10C140000000002090010000E859000898C1000894
:10C1500090010020B01A00005EAF00082113070410
:10C16000380D091E080540082609104008560A1314
:10C170001D043B08BE0596D8BC4010080430C842D8
:10C180000114020214130909120202C981938C0AD4
:08C19000024A015220000000E8
:04000005080050C1DE
:00000001FF
